TagPDF.com

c# tesseract ocr tiff: Running the Sample Microsoft OCR Application - C# Corner



c# zonal ocr













windows tiff ocr, .net ocr open source, activex ocr, ocr software open source linux, ocr software for asp net, perl ocr module, free ocr pdf to word mac, ocr sdk for c#.net, ocr vb net, ios coreml ocr, azure ocr pdf, ocr windows 7, asp.net core ocr, tesseract ocr library python, optical character recognition ocr in php using free api



google ocr api c#

How to implement and do OCR in a C# project? - Stack Overflow
15 Jan 2015 ... I wanted to know how to implement those open source OCR libraries to a C# project and how to use them. The link given as dup is not giving answers that I ...

c# ocr api open source


Web API test app for the OCR.SPACE Free OCR API as Visual Studio C# project. - A9T9/Free-OCR-API-CSharp.

Under Visual Basic 6 and previous versions, you can raise an error using the Err.Raise method. The Err object is still supported under Visual Basic .NET, so any code based on its Raise method will continue to work as before. However, you should throw your exceptions using the new Throw command to comply with the exception mechanism and make your code compatible with components written in other .NET languages.



tesseract ocr c# nuget


Create a new "Console Application" project, using C# or VB.NET ... Add the following code to create a private method to OCR, and export the data to the console.

microsoft ocr api c#


Mar 19, 2016 · Tesseract is an OCR library available for various different operating .... is a good open source option for optical character recognition in C# ...

The Remove and RemoveAt methods remove a single session variable. You can also delete all the session variables by using either the RemoveAll or the Clear method. The Count property returns the number of session variables. As with ASP, you can read the session identifier by means of the SessionID read-only property, and set or return the session timeout (in minutes) via the Timeout property. The IsNewSession property returns True if the session was created with the current request. The CodePage and LCID writeable properties let you decide the code page identifier and the locale identifier for the current session. The Keys property returns the collection of the names of all session variables:





modi ocr c#

C# Quick Start Guide - ABBYY Cloud OCR SDK
If you want to know how to work with OCR SDK in C# you should read the quick start guide with OCR SDK for C# .

c# ocr library

Deep Learning based Text Recognition ( OCR ... - Learn OpenCV
6 Jun 2018 ... In this tutorial, we will learn how to recognize text in images ( OCR ) using Tesseract's Deep Learning based LSTM engine and OpenCV .

) If a thread has hung the system by executing in an infinite loop at an IRQL of DPC/dispatch level or higher, you ll see the driver module in which it has become stuck in the stack trace of the !thread command The stack trace of the crash dump you get when you crash a system experiencing the Notmyfault hang bug looks like this: STACK_TEXT: f9e66ed8 f9b0d681 000000e2 00000000 00000000 nt!KeBugCheckEx+0x19 f9e66ef4 f9b0cefb 0069b0d8 010000c6 00000000 i8042prt!I8xProcessCrashDump +0x235 4 f9e66f3c 804ebb04 81797d98 8169b020 00010009 i8042prt!I8042KeyboardInterruptS ervice+0x21c 5 f9e66f3c fa12e34a 81797d98 8169b020 00010009 nt!KiInterruptDispatch+0x3d 6 WARNING: Stack unwind information not available Following frames may be wrong 7 ffdff980 8169b288 f9e67000 0000210f 00000004 myfault+0x34a 8 8054ace4 ffdff980 804ebf58 00000000 0000319c 0x8169b288 9 8054ace4 ffdff980 804ebf58 00000000 0000319c 0xffdff980 10 8169ae9c 8054ace4 f9b12b0f 8169ac88 00000000 0xffdff980 11 ...

Exam objectives in this chapter:

The values reappear along with the total for 2004. The values are stored in the writeback table and are now visible to anyone who accesses the cube. You can also write back values for a different scenario. Note

7

Understand common principles and considerations of performance test execution. Understand the common activities of performance test execution.

abbyy ocr c#

Extracting Text from an Image Using Tesseract in C# - CodeGuru
26 Feb 2019 ... Tesseract engine optical character recognition ( OCR ) is a technology used to convert scanned paper documents, PDF files, and images to searchable text data.

google ocr api c#


Please note that, our OCR SDK does not support directly importing PDF file. So, in the following C# demos, PDF documents will be firstly converted to Tiff image ...

DATA: Slot 0, Offset 0x60, Length 273, DumpStyle BYTE Record Type = PRIMARY_RECORD Record Attributes = NULL_BITMAP VARIABLE_COLUMNS Memory Dump @0x61C4C060 00000000: 00000010: 00000020: 00000030: ... 000000F0: 00000100: 00000110: 0...AAA{........ ....XXXXXXXXXXXX XXXXXXXXXXXXXXXX XXXXXXXXXXXXXXXX ... 58585858 58585858 58585858 58585858 XXXXXXXXXXXXXXXX 58585858 58585858 58585858 58584142 XXXXXXXXXXXXXXAB 43 C 30000900 0e011101 58585858 58585858 4141417b 58585858 58585858 58585858 000500e4 58585858 58585858 58585858 03000e01 58585858 58585858 58585858

The top few lines of the stack trace reference the routines that execute when you type the i8042 port driver s crash key sequence The presence of the Myfault driver indicates that it might be responsible for the hang Another command that might be revealing is !locks, which dumps the status of all executive resource locks By default, the command lists only resources that are under contention, which means that they are both owned and have at least one thread waiting to acquire them Examine the thread stacks of the owners with the !thread command to see what driver they might be executing in Sometimes you will find that the owner of one of the locks is waiting for an IRP to complete (a list of IRPs related to a thread is displayed in the !thread output) In these cases.

Given a choice, select the binary sort order. I have often found this to perform slightly better than the other sort orders, though not by much.

The OleDbTransaction object exposes a Begin method, which lets you start a transac; tion that s nested in the current transaction. The Begin method takes an optional isola; tion level and returns another OleDbTransaction object:

Version 2 certificate templates allow users with Write permission to change any attribute. The following sections detail modifications that can be made to version 2 certificate templates on a tab-by-tab basis.

Three types of objects are stored in tempdb: user objects, internal objects, and the version store, used primarily for snapshot isolation.

The TABLOCK option forces DBCC CHECKDB to take database and table locks to obtain its transactionally consistent view of the database (that is, the consistency checks are performed of ine and concurrent activity may be blocked). The locking behavior when this option is speci ed was described earlier in this chapter.

ps_3_0

c# zonal ocr


To get OCR in C# Console- Wpf- or WinForms-App: run on a modern Windows Version (e.g.: Win10); add nuget UwpDesktop; add the following code: var engine ...

c# read ocr pdf


Aug 4, 2015 · Microsoft OCR Library is for Windows Runtime app. And there is no direct way to use in Windows Form application. Following link has few ...












   Copyright 2021.